:0200000480007A
:10000000ADA8010001000100010001000100010094
:10001000232E11FE232C51FE232A61FE232871FE7C
:100020002326A1FE2324B1FE2322C1FE2320D1FEDC
:10003000232EE1FC232CF1FC232A01FD232811FDB2
:100040002326C1FD2324D1FD2322E1FD2320F1FD40
:100050003971AD28F250E2525253C2533255A25573
:10006000125682567247E2475248C248324EA24E5A
:10007000124F824F2161730020309741000093811D
:1000800061C2176100001301E1441385C1819765C6
:100090000000938565036306B50023200500110564
:1000A000DDBF173500001305A53F7111973500001E
:1000B0009385053F6308B500144111052AC0829657
:0C00C0000245EDB71101EF20704001A0D7
:1000CC00828003C75183930710046303F700828077
:1000DC001C4103A7C183A507998F1CC1828003A66D
:1000EC00418409C6184218C103A6418483A5C18363
:1000FC00310629456F00806D41114AC083A74184A8
:10010C0022C40041984326C283AE470003AE870049
:10011C0003A3070183A8470103A887018C53D0537D
:10012C00945706C6AA84C84FDC5718C0984048CCD0
:10013C005CD42322D40195472324C40123286400D2
:10014C00232A1401232C04010CD050D014D4DCC469
:10015C005CC418C0228561375C40B1CF9C40B24072
:10016C00224483AF070003AF470083AE870003AE82
:10017C00C70003A3070183A8470103A88701CC4F3D
:10018C009053D4539857DC5723A0F40123A2E401D5
:10019C0023A4D40123A6C40123A8640023AA140118
:1001AC0023AC0401CCCC90D0D4D098D4DCD402496C
:1001BC0092444101828088449947930584005CC431
:1001CC00EF00006D83A7418448441306C4009C4390
:1001DC00B24092441CC022440249A94541016F001F
:1001EC00E05E83C7518383A681839387F7FB93B724
:1001FC001700D58F23ACF18213072004238AE182E8
:10020C00828013071004A38AE18223AC01828280CE
:10021C0035711305000306CF22CDE2DCEED626CBDA
:10022C004AC94EC752C556C35AC1DEDEE6DAEAD811
:10023C00EF00E07423A0A18413050003EF002074E9
:10024C0083A7018423A2A1841CC189471CC5B7358F
:10025C000080930780025CC57D46938545CE2322A2
:10026C0005004105EF00D001373700809307C72404
:10027C00032EC72403A3470083A8870003A8C70045
:10028C008C4BD04B944F03D7C70183C7E701B73DC5
:10029C000080231EE102230FF10213874D5BA94757
:1002AC002945232EF76472D01AD246D442D62ED8C2
:1002BC0032DA36DCEF00807B37350080130545D011
:1002CC00EF0060782945EF00607A83A7018363868D
:1002DC00074C37350080130545D3EF00C076294510
:1002EC00EF00C07837350080130505D9EF00406B5F
:1002FC002945EF00A077373500809305800C130556
:10030C0085DCEF00E069EF0000773734008083274D
:10031C00C426373D0080832BCD283EC423A6A18262
:10032C0085491304C4268944E93D653D8347E401AE
:10033C005048032E4400032384008328C400032860
:10034C000401144C0357C401A24E230FF1048C007A
:10035C0085470810B2CA3ECE26CAF6C0F2C29AC46D
:10036C00C6C6C2C8B6CC231EE104DD2152461335E5
:10037C00150023ACA18263C0C40293172600B29768
:10038C00F51732858D4530083ECC8921524605063D
:10039C0032CAE3D4C4FEE2461385C18493854D5B17
:1003AC00152903A54184930A10040D4AB13303C7E0
:1003BC00418393070004930CCD2863F1E702568523
:1003CC00930530049529F24713871A00630EF5360E
:1003DC0083C74183937AF70FE3F357FFD2455285D6
:1003EC008509EF20A07BE24A2AC6D685EF20407D06
:1003FC002A8A480852CAF1319307900CE396F9F215
:10040C00EF00606723A4A18237350080130585DFD8
:10041C00EF0060632945EF006065373500801305F8
:10042C0085E0EF0040622945EF00406483A5C1835D
:10043C0037350080130505E437340080EF00405653
:10044C0095451305C4E5EF00A05583A58183373589
:10045C000080130585E7EF00A05485451305C4E51E
:10046C00EF00005483C5518337350080130545E9EF
:10047C00052BB734008093051004138504EB0D2372
:10048C0083C54183373500801305C5EC112B9305CB
:10049C002004138504EB29239387C1848C533735AF
:1004AC000080130585EEED299D451305C4E5CD2986
:1004BC00B73700809387475B83A5C76537350080C6
:1004CC00130545F0F12937350080130505F2EF00CF
:1004DC008057373500801305C5F4EF00C05683A74D
:1004EC004184B73D008013858DF58C43B73C00806B
:1004FC00B73B0080752137350080130545F7EF00B9
:10050C00805483A7418413854CFA373B0080CC433D
:10051C00B739008037390080612181451305C4E566
:10052C00412183A7418413850BFC8C479529894570
:10053C001305C4E5B52183A741841305CBFDCC4736
:10054C008521C5451305C4E5A12983A541841385DF
:10055C0089FFC105B12113054901F521373500800B
:10056C0013058504CD2183A7018413858DF58C4358
:10057C0005293735008013058505F12183A70184F2
:10058C0013854CFACC43292981451305C4E5092967
:10059C0083A7018413850BFC8C4719218545130512
:1005AC00C4E5FD2E83A701841305CBFDCC47CD2ECE
:1005BC00C9451305C4E5ED2683A50184138589FF80
:1005CC00C105F92E13054901BD29D24537350080E7
:1005DC0013058509F12695451305C4E5D126B247C7
:1005EC00373500801305450BB38A574193973A0072
:1005FC00B38A5741B3854A416526B5451305C4E511
:10060C004526E245373500801305050D512E9D45D5
:10061C001305C4E57126F245373500801305C50E68
:10062C00412685451305C4E5A52E373500800C10F1
:10063C0013058510B5263735008013054512212189
:10064C00373500808C0013058515992E37350080C1
:10065C0013054517CD2E2945112903A7C18283A562
:10066C0081829307301F998D23A2B18263DFB71269
:10067C003735008013050520252603A54182EF2080
:10068C0060152A84EF204027B737008003A6074A5D
:10069C0083A6474AEF001066B737008003A6874A47
:1006AC0083A6C74AEF000064EF20C03523A0A182C7
:1006BC00B737008003A5074BA285EF10A05223AEDD
:1006CC00A1803735008013054521D92C03A5418223
:1006DC00EF204010B7370080AA8503A5474BEF10D9
:1006EC0060502A84EF200008AA84EF20A00EAA856F
:1006FC002285EF10B03FB737008083A5874BEF10F2
:10070C00F007EF2020062A8437350080A6851305D4
:10071C0045247924A54763D7870A37350080A285FD
:10072C0013058524B52C29459126FA406A44DA44F0
:10073C004A49BA492A4A9A4A0A4BF65B665CD65C25
:10074C00465DB65D0D6182806C080145912203AE59
:10075C004C0003A38C0083A8CC0003A80C0103A5B8
:10076C004C0183A58C0103D6CC0103C7EC0183C7D4
:10077C004183850ADEC0F2C29AC4C6C6C2C8AACAE0
:10078C00AECC231EC104230FE10423AE318393FAB4
:10079C00FA0F4E8AE3F557C391B137350080130534
:1007AC0005D655242945D92435BE37350080130587
:1007BC00851A512C373500801305051E69242945EF
:1007CC007524A5B713050003552481BF0905AA9507
:1007DC000CC2828001114EC69309560026CA93940E
:1007EC00290022CC4AC806CEAA9432892E8423AC86
:1007FC00340794C0D4C04E859305800CEF20003A8A
:10080C000A09B3072501A297984B23AA370123ACF9
:10081C003701050798CB9C402A944A94056632947C
:10082C00232AF4FAF2406244154723AEE182D24403
:10083C004249B249056182801375F50F93F5F50FA6
:10084C006304B50001458280A38AA182054582809C
:10085C00411122C426C206C62A84AE8483C5340044
:10086C0003452400D13F7DF9A6852285F52C8147CF
:10087C006356A000294723AEE1828547B24022444B
:10088C0092443E8541018280791513351500828092
:10089C00411122C426C206C62A84AE84F53715C17E
:1008AC0080C085476304F40205C80947630DE40260
:1008BC0091476313F40098C0B24022449244410122
:1008CC0082808D479CC08547E310F4FE03A7C1834B
:1008DC009307400663DFE700B240224423A00400E4
:1008EC00924441018280B24022449CC09244410116
:1008FC008280B24022448D479CC092444101828048
:10090C00411122C406C62A840345050011C50504FD
:10091C00B12A0345040065FDB240224441018280A6
:10092C00B1A2797126D206D622D44AD0AA846342C7
:10093C0005040A894A8429A8EF20C03093070503CF
:10094C0005042685A945A30FF4FEEF206027AA8491
:10095C00A9452685F5F0E30124FF7D140345040029
:10096C00C137E31C24FFB250225492540259456102
:10097C0082801305D0026D37B30490405DBF03A78E
:10098C008184B307A7003765008023A4F184130585
:10099C0045CC930600403A9563D3F60002908280D2
:1009AC005D7152CC06D622D426D24AD04ECE56CA2F
:1009BC002A8A03450500BEC25C182EDA32DC36DE0C
:1009CC00BAC0C2C4C6C63EC61DC10144930A500279
:1009DC00930430061309300793094006630255034C
:1009EC0081370504B3078A0003C5070065F9B250C7
:1009FC00225492540259F249624AD24A616182806D
:100A0C00930614003307DA0031A063822703638650
:100A1C00370385068347070036840507F9D3E39629
:100A2C0097FEB247884391073EC6DD3D5DBFB24796
:100A3C00884391073EC6E9356DB7B24788439107A5
:100A4C003EC6C53579BF411122C406C62A8403456A
:100A5C00050011C5050419280345040065FD294549
:100A6C003120B2402244014541018280B70710F089
:100A7C0023A0A7F08280B70710F003A507F18280AE
:100A8C00B3C7A50093F737003307C500639607007B
:100A9C009307300063E4C70293070500636CE5001D
:100AAC006780000083C605009387170093851500A7
:100ABC00A38FD7FEE3E8E7FE67800000937735004D
:100ACC0063920708930705009376C7FF138606FE0B
:100ADC0063F6C70883A3050083A2450083AF850096
:100AEC0003AFC50083AE050103AE450103A3850129
:100AFC0083A8C501938545029387470203A8C5FFC8
:100B0C0023AE77FC23A057FE23A2F7FF23A4E7FF15
:100B1C0023A6D7FF23A8C7FF23AA67FE23AC17FF82
:100B2C0023AE07FF6FF0DFFA83C60500938717002B
:100B3C0093851500A38FD7FE93F63700E39606FE38
:100B4C006FF09FF8930705006FF01FFF03A60500D9
:100B5C00938747009385450023AEC7FEE3E8D7FE95
:100B6C00E3EAE7F4678000003367B5009303F0FF16
:100B7C001377370063100710B7877F7F9387F7F7DA
:100B8C000326050083A60500B372F6003363F60056
:100B9C00B382F200B3E26200639272106316D6085D
:100BAC000326450083A64500B372F6003363F600B6
:100BBC00B382F200B3E26200639E720C6316D60637
:100BCC000326850083A68500B372F6003363F60016
:100BDC00B382F200B3E262006398720C6316D6041F
:100BEC000326C50083A6C500B372F6003363F60076
:100BFC00B382F200B3E262006392720C6316D60207
:100C0C000326050183A60501B372F6003363F600D3
:100C1C00B382F200B3E26200639C720A13054501D1
:100C2C0093854501E30ED6F413170601939706013D
:100C3C00631EF7001357060193D706013305F740DF
:100C4C009375F50F63900502678000001357070139
:100C5C0093D707013305F7409375F50F639405009F
:100C6C00678000001377F70F93F7F70F3305F74002
:100C7C00678000000346050083C6050013051500B8
:100C8C00938515006314D600E31606FE3305D64093
:100C9C00678000001305450093854500E31CD6FCD6
:100CAC0013050000678000001305850093858500FF
:100CBC00E312D6FC13050000678000001305C50085
:100CCC009385C500E318D6FA130500006780000071
:100CDC001305050193850501E31ED6F813050000E5
:100CEC0067800000130101FB23248104232C4103A2
:100CFC003704100013DA450123202105232E31037C
:100D0C00232A5103232481031304F4FF2326110403
:100D1C0023229104232861032326710323229103A8
:100D2C002320A103232EB101137AFA7F13090500A6
:100D3C00130C0600938A06003374B40093D9F501A2
:100D4C0063060A0A9307F07F6304FA101314340045
:100D5C00B70780003364F400135BD501336B8B0051
:100D6C0093143500130A1AC0930B000013D54A01D3
:100D7C00370910001309F9FF1375F57F3379590101
:100D8C0093050C0093DAFA01630205109307F07FC8
:100D9C006302F51637048000131939003369890092
:100DAC001354DC013364240193153C00130515C066
:100DBC009307000013972B003367F7001307F7FF17
:100DCC009306E00033C95901330AAA4063E0E616E2
:100DDC00972600009386064D131727003307D7007C
:100DEC00032707003307D70067000700336BA40005
:100DFC00630E0B066300040413050400EF109067E8
:100E0C00930755FF1307C001634CF702130BD00176
:100E1C00930485FF330BFB4033149400335B69015F
:100E2C00336B8B00B3149900130AD0C0330AAA4059
:100E3C006FF09FF3EF101064130505026FF05FFC69
:100E4C00130485FD331B8900930400006FF0DFFD54
:100E5C00336BA40063040B0293040500130B040012
:100E6C00130AF07F930B30006FF05FF093040000D7
:100E7C00130A0000930B10006FF05FEF9304000057
:100E8C00130AF07F930B20006FF05FEE336489013F
:100E9C00630E04066300090413050900EF10905D4E
:100EAC00930755FF1307C001634EF7021304D001DB
:100EBC00930585FF3304F4403319B90033548C0087
:100ECC0033642401B315BC001307D0C03305A7400D
:100EDC006FF01FEE13050C00EF10D059130505022F
:100EEC006FF01FFC130485FD33148C009305000078
:100EFC006FF09FFD3364890163020402130409003F
:100F0C001305F07F930730006FF0DFEA93050000C4
:100F1C0013050000930710006FF0DFE99305000044
:100F2C001305F07F930720006FF0DFE86366640120
:100F3C0063128B4863E0B4489316FB0113D714007B
:100F4C00139CF401135B1B00B3E4E6001314840040
:100F5C0093DC8501B3EC8C0093DA0C0193970C01B4
:100F6C0093D70701139D850013050B0093850A0089
:100F7C002322F100EF10504593050500930B05005B
:100F8C0013950C0113550501EF1050411304050086
:100F9C0093850A0013050B00EF10904713150501FC
:100FAC0013D704013365A70093890B00637E85007A
:100FBC00330595019389FBFF636895016376850082
:100FCC009389EBFF330595013304854093850A0023
:100FDC0013050400EF10503F93050500930B05001B
:100FEC0013950C0113550501EF10503B130B050025
:100FFC0093850A0013050400EF109041939D0401A2
:10100C001315050193DD0D01B3EDAD0013870B0036
:10101C0063FE6D01B38D9D011387FBFF63E89D019A
:10102C0063F66D011387EBFFB38D9D019396090158
:10103C00B7040100B3E6E600B38D6D41138BF4FFEA
:10104C0033F76601337B6D011305070093050B0025
:10105C0013D406012326D1002324E100EF10103411
:10106C002322A10093050B0013050400EF1010338D
:10107C00935B0D019309050093850B001305040088
:10108C00EF10D031032781001304050013850B00EA
:10109C0093050700EF10903003264100330535010E
:1010AC008326C100135706013307A7006374370169
:1010BC0033049400370501001305F5FF9354070121
:1010CC00B379A700939909013376A600B384840001
:1010DC00B389C90063E89D001384060063949D04E2
:1010EC0063723C05330CAC013337AC013307970109
:1010FC00B38DED001384F6FF63E6BC016394BC036F
:10110C006362AC0363E69D00639EB401637C3C01A7
:10111C00330CAC013337AC01330797011384E6FF72
:10112C00B38DED00B3093C41B3849D40B3373C0112
:10113C00B384F4409305F0FF63889C1A93850A00EE
:10114C0013850400EF105028930505002324A100FB
:10115C0013950C0113550501EF1050242322A10007
:10116C0093850A0013850400EF10902A83268100D2
:10117C00032741001315050193D7090133E5A70097
:10118C00938D0600637EE50033059501938DF6FF84
:10119C00636895016376E500938DE6FF3305950151
:1011AC00B304E54093850A0013850400EF10D021A9
:1011BC00930505002322A10013950C01135505017D
:1011CC00EF10D01D130C050093850A001385040045
:1011DC00EF10102493990901032741001315050101
:1011EC0093D9090133E5A90093070700637E8501B4
:1011FC00330595019307F7FF6368950163768501C5
:10120C009307E7FF3305950193940D01B3E4F400C4
:10121C009397040193D7070193050B00B3098541FC
:10122C00138507002322F10093DD0401EF10101742
:10123C0093050B00930A050013850D00EF10101693
:10124C00130C050093850D0013850B00EF10101582
:10125C0083274100130B050013850B0093850700B2
:10126C00EF10D0133305850193D70A013385A700FE
:10127C0063768501B7070100330BFB00B70601004D
:10128C009386F6FF935705013377D50013170701A3
:10129C00B3FADA00B38767013307570163E8F90043
:1012AC00938504006390F9046300070433853C01C3
:1012BC009385F4FF636495036366F5006314F5028C
:1012CC006370ED0293161D0033BDA601B30C9D0196
:1012DC009385E4FF33059501138D06006314F50027
:1012EC006304A70193E515001307FA3F6352E0125C
:1012FC0093F775006380070293F7F500930640009F
:10130C00638AD70093864500B3B5B6003304B400A6
:10131C00938506009317740063DA0700B70700FF84
:10132C009387F7FF3374F40013070A409307E07FA9
:10133C0063C2E71A9317D40193D53500B3E7B7000E
:10134C0013543400B70610009386F6FF3374D400A0
:10135C00B70610801377F77F9386F6FF13174701B4
:10136C003374D4001319F9013364E4003367240196
:10137C008320C10403248104832441040329010430
:10138C008329C103032A8103832A4103032B01030D
:10139C00832BC102032C8102832C4102032D0102F9
:1013AC00832DC10113850700930507001301010567
:1013BC0067800000130AFAFF130C00006FF01FB9CE
:1013CC001389090013040B009385040093870B0009
:1013DC00130720006380E710130730006382E70EC9
:1013EC0013071000E392E7F01304000093070000CA
:1013FC006F00400913890A006FF09FFD3704080045
:10140C009305000013090000930730006FF05FFC98
:10141C0093061000B386E64093078003E3C6D7FC1F
:10142C009307F00163C4D706130AEA41B3174401CA
:10143C0033D7D500339A4501B3E7E700333A40017F
:10144C00B3E747013354D40013F777006300070266
:10145C0013F7F70093064000630AD7001387470081
:10146C00B337F7003304F400930707001317840015
:10147C00634A07061317D40193D73700B367F700F5
:10148C0013543400130700006FF0DFEB930710FECA
:10149C00B387E74013070002B357F40013050000AD
:1014AC006386E600130AEA4333154401336AB50038
:1014BC00333A4001B3E74701130400006FF0DFF843
:1014CC0037040800930700001307F07F130900008E
:1014DC006FF05FE713040000930700001307F07F21
:1014EC006FF05FE613040000930700001307100071
:1014FC006FF05FE5130101FA232C810423263105DB
:10150C003704100093D94501232A91042320610547
:10151C00232E7103232C81031304F4FF232E1104B7
:10152C00232821052324410523225105232A910335
:10153C002328A1032326B10393F9F97F9304050013
:10154C00930B0600138C06003374B40013DBF50107
:10155C006388090A9307F07F6386F91037098000C6
:10156C0013143400336424011359D50133698900F1
:10157C00131D3500938919C0930C000013554C01B1
:10158C00370A1000130AFAFF1375F57F337A8A01B4
:10159C0093840B00135CFC01630405109307F07F2C
:1015AC006304F51637048000131A3A00336A8A0074
:1015BC0013D4DB013364440193943B00130515C031
:1015CC009307000013972C003367F700B389A90029
:1015DC001307F7FF9306E000B34B8B01938A1900B6
:1015EC0063E0E61697260000938686CF1317270034
:1015FC003307D700032707003307D700670007001E
:10160C003369A400630E0906630004041305040087
:10161C00EF104066930755FF1307C001634CF702A8
:10162C001309D001130D85FF3309F9403314A401BC
:10163C0033D9240133698900339DA4019309D0C0A7
:10164C00B389A9406FF05FF3EF10C0621305050278
:10165C006FF05FFC130985FD33992401130D000015
:10166C006FF0DFFD3369A40063040902130D05005C
:10167C00130904009309F07F930C30006FF01FF0F6
:10168C00130D000093090000930C10006FF01FEF76
:10169C00130D00009309F07F930C20006FF01FEEE8
:1016AC0033647A01630E040663000A0413050A000E
:1016BC00EF10405C930755FF1307C001634EF70210
:1016CC001304D001930485FF3304F440331A9A00B9
:1016DC0033D48B0033644401B3949B009307D0C084
:1016EC003385A7406FF0DFED13850B00EF108058AA
:1016FC00130505026FF01FFC130485FD33948B005A
:10170C00930400006FF09FFD33647A0163020402BE
:10171C0013040A001305F07F930730006FF09FEA63
:10172C009304000013050000930710006FF09FE96D
:10173C00930400001305F07F930720006FF09FE8DF
:10174C0037070100130AF7FF135C0D0193DD040149
:10175C00337D4D01B3F4440193050D001385040052
:10176C002328E100EF108043930C050093850400BF
:10177C0013050C00EF1080422326A10093850D0069
:10178C0013050C00EF108041130B050093050D00A1
:10179C0013850D00EF1080408326C10093D70C01F8
:1017AC003305D5003385A7006376D50003270101E7
:1017BC00330BEB009356050133754501B3FC4C011B
:1017CC0013150501B3079501935C040133744401AF
:1017DC0093050D0013050400232AD1002326F100E4
:1017EC00EF10C03B2328A1009305040013050C0047
:1017FC00EF10C03A130A050093850C0013050C007A
:10180C00EF10C039130C050093050D0013850C0067
:10181C00EF10C03803270101330545018326410130
:10182C00935707013385A70063764501B70701007D
:10183C00330CFC003706010093570501338C8701EC
:10184C009307F6FF337AF5003377F700131A0A0182
:10185C00135D0901330AEA003379F9003387460135
:10186C0093050900138504002328E100232EC100F1
:10187C00EF10C03293850400232CA10013050D003A
:10188C00EF10C031232AA10093050D0013850D0024
:10189C00EF10C030930405009305090013850D006B
:1018AC00EF10C02F83264101032781013305D5009A
:1018BC00935707013385A7006376D5000326C10132
:1018CC00B384C400B70601009387F6FF935D05014E
:1018DC00B3849D00B37DF5003377F70093050900C1
:1018EC0013050400939D0D01B38DED00232CD10045
:1018FC00EF10C02A93050400232AA10013050D0044
:10190C00EF10C02993050D001304050013850C007E
:10191C00EF10C028130D05009305090013850C006A
:10192C00EF10C027032741013305850093570701AA
:10193C003385A7006376850083268101330DDD0096
:10194C0083270101B70601009386F6FF330BFB00DA
:10195C00B377D5003377D70093970701B387E700A8
:10196C00333A4B01B387870133844701330BBB01F7
:10197C0033079400B33DBB01B306B70133BC8701F9
:10198C0033344401935705013337970033648C008B
:10199C00B3BDB6013304F400B36DB7013304B40125
:1019AC003304A40193D77601131494003364F40028
:1019BC008327C10093149B00135B7B01B3E4F400F9
:1019CC00B334900093979600B3E46401B3E4F4004D
:1019DC009317740063D2071293D7140093F4140076
:1019EC00B3E497009317F401B3E4F4001354140018
:1019FC001387FA3F6356E01093F774006380070275
:101A0C0093F7F40093064000638AD7009387440051
:101A1C00B3B49700330494009384070093177400B5
:101A2C0063DA0700B70700FF9387F7FF3374F400FE
:101A3C0013870A409307E07F63C6E71893DA3400F4
:101A4C009314D401B3E4540113543400B7071000B9
:101A5C009387F7FF3374F4009377F77F3707108081
:101A6C001307F7FF939747013374E400939BFB0133
:101A7C003364F400B36774018320C105032481052A
:101A8C001385040003290105832441058329C1041E
:101A9C00032A8104832A4104032B0104832BC103F1
:101AAC00032C8103832C4103032D0103832DC102DD
:101ABC00938507001301010667800000930B0B0050
:101ACC001304090093040D0093870C0013072000E6
:101ADC00638AE70E13073000638CE70C13071000C2
:101AEC00E398E7F013040000930400006F008008F3
:101AFC00930B0C006FF09FFD938A09006FF05FEF62
:101B0C0093061000B386E64093078003E3CCD7FC22
:101B1C009307F00163C4D706938AEA41B3175401C3
:101B2C0033D7D400B3945401B3E7E700B334900037
:101B3C00B3E497003354D40093F774006380070226
:101B4C0093F7F40013074000638AE700938744007F
:101B5C00B3B4970033049400938407009317840064
:101B6C0063CA07069317D40193D43400B3E49700E7
:101B7C0013543400130700006FF05FED930710FE51
:101B8C00B387E74013060002B357F40013070000B5
:101B9C006386C600938AEA4333175401B3649700F3
:101BAC00B3349000B3E49700130400006FF0DFF837
:101BBC0037040800930400001307F07F930B000018
:101BCC006FF0DFE813040000930400001307F07FAC
:101BDC006FF0DFE7130400009304000013071000FC
:101BEC006FF0DFE6130101FD23229102232A51013C
:101BFC0093547501B70A8000232021032328610127
:101C0C00938AFAFF2326110223248102232E310109
:101C1C00232C4101232671012324810193F4F40F19
:101C2C00138B0500B3FAAA001359F5016388040855
:101C3C009307F00F6384F40A939A3A00B7070004F1
:101C4C00B3EAFA00938414F8930B000013557B014C
:101C5C00370480001304F4FF1375F50F337464011B
:101C6C00135BFB01630C05089307F00F6308F50A7F
:101C7C0013143400B70700043364F400130515F88B
:101C8C009307000013972B003367F7001307F7FF38
:101C9C009306E000B3496901338AA44063E0E60A85
:101CAC009716000093868667131727003307D70013
:101CBC00032707003307D70067000700638A0A026F
:101CCC0013850A00EF00107B9307B5FF9304A0F86F
:101CDC00B39AFA00B384A4406FF01FF79304F00F8B
:101CEC00930B2000E3840AF6930B30006FF01FF681
:101CFC0093040000930B10006FF05FF5630A04026D
:101D0C0013050400EF0010779307B5FF3314F400AC
:101D1C009307A0F83385A7406FF09FF61305F00FDB
:101D2C0093072000E30004F6930730006FF09FF553
:101D3C0013050000930710006FF0DFF4131B540021
:101D4C0063F68A12130AFAFF13090000935B0B0166
:101D5C003704010093850B001304F4FF13850A006C
:101D6C00EF00906633748B0093050500130C05008F
:101D7C0013050400EF0090629304050093850B009B
:101D8C0013850A00EF00D0681359090113150501DA
:101D9C003365A90013090C00637E950033056501BA
:101DAC001309FCFF63686501637695001309ECFF6A
:101DBC0033056501B304954093850B00138504002E
:101DCC00EF00906093050500130C0500130504004B
:101DDC00EF00D05C930A050093850B00138504007B
:101DEC00EF0010631315050113040C00637E5501FD
:101DFC00330565011304FCFF6368650163765501C7
:101E0C001304ECFF33056501131909013305554122
:101E1C00336989003335A0003364A9001307FA072E
:101E2C006350E00A93777400638A07009377F40099
:101E3C00930640006384D7001304440093174400B6
:101E4C0063DA0700B70700F89387F7FF3374F400E1
:101E5C0013070A089307E00F1354340063D2E70CFE
:101E6C00130400001307F00F6F00800B1399FA0195
:101E7C0093DA1A006FF09FED9309090013840A009E
:101E8C0093870B0013072000E38CE7FC130730004B
:101E9C006382E70813071000E392E7F813040000CD
:101EAC00130700006F00C00793090B006FF09FFD34
:101EBC003704400093090000930730006FF09FFC3B
:101ECC0093071000B387E7401307B001E348F7FC12
:101EDC001305EA09B357F4003314A400333480001B
:101EEC0033E4870093777400638A07009377F400D8
:101EFC00130740006384E700130444009317540055
:101F0C0013543400E3DE07F8130400001307100029
:101F1C006F000001370440001307F00F9309000015
:101F2C00370580001305F5FF3374A4003705808056
:101F3C001305F5FF1377F70F3374A400131777010C
:101F4C001395F9013364E4003365A4008320C102C6
:101F5C000324810283244102032901028329C10144
:101F6C00032A8101832A4101032B0101832BC10028
:101F7C00032C81001301010367800000130101FD94
:101F8C002322910223202103B704800013597501E9
:101F9C00232E3101232671019384F4FF2326110291
:101FAC0023248102232C4101232A5101232861017E
:101FBC0023248101232291011379F90F938B0500BE
:101FCC00B3F4A4009359F501630A09089307F00FC1
:101FDC006306F90A93943400B7070004B3E4F400E1
:101FEC00130919F8130B000013D57B01370480007B
:101FFC001304F4FF1375F50F3374740193DBFB01B9
:10200C00630E05089307F00F630AF50A13143400E6
:10201C00B70700043364F400130515F893060000A9
:10202C0093172B00B3E7D7003309A9009387F7FF69
:10203C001307E00033CA7901930A19006360F70AA9
:10204C00171700001307473193972700B387E70052
:10205C0083A70700B387E70067800700638A040241
:10206C0013850400EF0010419307B5FF1309A0F886
:10207C00B394F4003309A9406FF0DFF61309F00FA5
:10208C00130B2000E38204F6130B30006FF0DFF526
:10209C0013090000130B10006FF01FF5630A040204
:1020AC0013050400EF00103D9307B5FF3314F40043
:1020BC009307A0F83385A7406FF05FF61305F00F78
:1020CC0093062000E30E04F4930630006FF05FF5E6
:1020DC0013050000930610006FF09FF4370C0100FD
:1020EC00130BFCFF93DB0401935C0401B3F4640158
:1020FC00337464019305040013850400EF00102A67
:10210C00930504009309050013850B00EF001029BB
:10211C001304050093850C0013850B00EF001028A9
:10212C00930B05009385040013850C00EF0010271A
:10213C003305850093D709013385A70063748500A7
:10214C00B38B8B01B377650193970701B3F96901E1
:10215C00B3873701139467003334800093D7A701FA
:10216C0013550501B367F4003304750113146400AF
:10217C003364F4009317440063D6070E935714008E
:10218C001374140033E487001387FA076350E00ECE
:10219C0093777400638A07009377F40093064000EA
:1021AC006384D700130444009317440063DA0700D8
:1021BC00B70700F89387F7FF3374F40013870A0806
:1021CC009307E00F63C4E710935734006F000003CC
:1021DC00138A09001384040093060B009307200054
:1021EC006386F60E93073000638AF60C1306100014
:1021FC009307000013070000E398C6F8370480002B
:10220C001304F4FF37058080B3F787001305F5FF3F
:10221C008320C102032481021377F70FB3F7A700C1
:10222C00131777011315FA01B3E7E7008324410272
:10223C00032901028329C101032A8101832A410157
:10224C00032B0101832BC100032C8100832C410043
:10225C0033E5A7001301010367800000138A0B000C
:10226C006FF0DFF7930A09006FF01FF2930710006D
:10227C00B387E7401307B0016340F706938AEA0976
:10228C00B357F400331454013334800033E4870023
:10229C0093777400638A07009377F4001307400068
:1022AC006384E700130444009317540063CA0702C5
:1022BC0093573400130700006FF05FF4B70740002A
:1022CC001307F00F130A00006FF05FF39307000081
:1022DC001307F00F6FF09FF2930700006FF09FFD54
:1022EC0093070000130710006FF05FF1B707800031
:1022FC009387F7FF130101FF33F7A700935675017E
:10230C0013D67501B3F7B7002322910023202101C6
:10231C0093F6F60F131837001376F60F23261100D9
:10232C00232481001307F00F9354F5011389060041
:10233C001305060093D5F501939737006314E60057
:10234C006394070093C515003387C640639A951AAA
:10235C006356E00A63160606639C07009307F00FAA
:10236C00638CF60493070800138506006F00C014F5
:10237C001307F7FF631E0702B387070113850600D7
:10238C0013975700635A0712130515001307F00F24
:10239C00630EE5323707007E93F617001307F7FF3D
:1023AC0093D71700B3F7E700B3E7D7006F00C0105F
:1023BC001306F00F639EC600930708006F004007DA
:1023CC001306F00FE38AC6FE37060004B3E7C70016
:1023DC001306B0016356E600930710006FF0DFF9A7
:1023EC00130600023306E640B3D5E700B397C700E7
:1023FC00B337F000B3E7F5006FF01FF86300070880
:10240C00639C0602631808001307F00F6316E60AB4
:10241C006F0000029306F0FF6316D700B387070125
:10242C006FF01FF69306F00F1347F7FF6310D602F9
:10243C001305F00F6F0040089306F00FE30AD6FE69
:10244C00B70600043307E0403368D8009306B001A8
:10245C0063D6E600130710006F00C001930600025C
:10246C003356E8003387E6403317E8003337E00093
:10247C003367E600B387E7006FF09FF01385160013
:10248C001376F50F130710006342C7066394060416
:10249C00130500006302080263860722B387070155
:1024AC0013975700635A0700370700FC1307F7FF11
:1024BC00B3F7E7001305100013F77700630A072042
:1024CC0013F7F700930640006304D7209387470067
:1024DC006F000020E30E08F4E38007EEB70700025C
:1024EC001305F00F930400006F00801E1307F00F0C
:1024FC00630EE51C3307F800935717006FF0DFFBF2
:10250C006350E00863160604E38A07E41307F7FF39
:10251C0063140702B307F84013850600139757009E
:10252C00E35C07F8370400041304F4FF33F487006A
:10253C00130905006F0080131306F00FE38EC6E637
:10254C001306B0016350E602930710006FF09FFC76
:10255C001306F00FE382C6E637060004B3E7C700A4
:10256C006FF01FFE13060002B3D5E7003307E640F9
:10257C00B397E700B337F000B3E7F5006FF09FF9BE
:10258C0063020708639E0602631808001307F00F26
:10259C00938405006FF09FE79306F0FF6318D70054
:1025AC00B3870741938405006FF05FF79306F00F34
:1025BC001347F7FF6310D602938405006FF05FE7B3
:1025CC009306F00FE30AD6FEB70600043307E0408B
:1025DC003368D8009306B00163D6E60013071000E9
:1025EC006F00C001930600023356E8003387E640C3
:1025FC003317E8003337E0003367E600B387E74072
:10260C006FF05FFA138716001377F70F130610009D
:10261C006344E604639C060263180800639807127F
:10262C00130500006FF01FEC638607123307F840A8
:10263C0093165700B387074163CA06109307070028
:10264C0063100706930700006FF09FFDE31608E880
:10265C00E39407F66FF09FE83304F8401317540027
:10266C006354070433840741938405001305040065
:10267C00EF0040601305B5FF3314A400634A250333
:10268C00330525411305150013070002B357A400A9
:10269C003305A7403314A40033348000B3E787001C
:1026AC00130500006FF05FE1E30E04F86FF01FFC00
:1026BC00B70700FC9387F7FF3305A940B377F40005
:1026CC006FF09FDF930708006FF01FDF9307000088
:1026DC0013975700635E0700130515001307F00FDF
:1026EC00630EE506370700FC1307F7FFB3F7E700A7
:1026FC001307F00F93D737006318E50063860700C4
:10270C00B707400093040000370780001307F7FF5A
:10271C001375F50FB3F7E7001317750137058080B4
:10272C008320C100032481001305F5FF33F5A700B6
:10273C009394F4013365E50033659500032901009A
:10274C00832441001301010167800000938405007C
:10275C006FF01FF5930708006FF09FF493070000CC
:10276C006FF01FF937068000135775019307F6FFBA
:10277C001377F70F9305E007B3F7A7009356F5010E
:10278C0063F6E5049305D00963FAE500370500808C
:10279C001345F5FF3385A6006780000033E5C700BD
:1027AC009307500963DCE7001307A7F63315E50020
:1027BC00638006023305A040678000009307600920
:1027CC003387E7403355E5006FF09FFE130500009B
:1027DC0067800000130101FF2326110023248100D0
:1027EC002322910063020510130405009354F50194
:1027FC00635405003304A04013050400EF00804728
:10280C009307E009B387A740130760096340F706F5
:10281C00130780006356A700130585FF3314A4002B
:10282C00370580001305F5FF93F7F70F3374A400F9
:10283C0013957701B70780809387F7FF3374F40003
:10284C00B70700803364A40093C7F7FF1395F40116
:10285C003374F4003365A4008320C1000324810089
:10286C0083244100130101016780000013079009C4
:10287C006350F702130750003307A7409306B501C6
:10288C003357E4003314D4003334800033648700AE
:10289C00130750006356A7001307B5FF3314E40069
:1028AC00370700FC1307F7FF937674003377E400C7
:1028BC00638A06001374F400930640006304D4008A
:1028CC00130747009316570063DC0600B70700FC9C
:1028DC009387F7FF3377F7009307F009B387A74087
:1028EC00135437006FF0DFF313040000930700005C
:1028FC00930400006FF0DFF293577501130101FF91
:10290C0093F7F70F232481001387170037048000F7
:10291C00232291001304F4FF232611001377F70FE1
:10292C00930610003374A4009354F50163D2E606A9
:10293C0013850738935734001314D401370710004C
:10294C001307F7FFB3F7E700370710801307F7FFFC
:10295C001375F57F13154501B3F7E70037070080B2
:10296C00B3E7A7001347F7FF1395F401B3F7E7009C
:10297C0033E7A7008320C100130504000324810062
:10298C0083244100930507001301010167800000B7
:10299C00639407046302040613050400EF00802D02
:1029AC009307A00063C2A7029307B000B387A740A8
:1029BC0013075501B357F4003314E4001307903890
:1029CC003305A7406FF09FF7930755FFB317F4003B
:1029DC00130400006FF09FFE93070000630A0400CD
:1029EC0093573400370708001314D401B3E7E700FA
:1029FC001305F07F6FF09FF49307000013050000A0
:102A0C006FF0DFF3370610001306F6FF3376B600CF
:102A1C0013D845019357D5011378F87F1316360058
:102A2C0033E6C7009307180093F7F77F930610005F
:102A3C0093D5F5011317350063D6F60A930608C82B
:102A4C009307E00F63C2D70C6340D008930790FE46
:102A5C0063C4F612B70780001305E0013366F60075
:102A6C003305D5409307F00163C8A702130828C8A3
:102A7C00B3170701B337F000331606013355A7001F
:102A8C00B3E7C700B367F5009306000013F77700B0
:102A9C00630007086F00C00E9307E0FFB386D740B2
:102AAC0093070002B356D600930800006306F500A6
:102ABC00130828CAB3180601B3E7E800B337F000CF
:102ACC00B3E7F6006FF05FFC131565003335A0001B
:102ADC00131636009357D7013366C500B367F6005B
:102AEC006FF0DFFAB367E60063160800B337F00047
:102AFC006FF09FF99306F00F638C070013163600E6
:102B0C00B70700026FF09FFD930700009306F00FCC
:102B1C0013975700635E0700938616001307F00F98
:102B2C00638AE606370700FC1307F7FFB3F7E700E5
:102B3C001307F00F93D737006398E60063860700FE
:102B4C00B707400093050000370580001305F5FF1B
:102B5C00B3F7A700370580801305F5FF93F6F60F42
:102B6C0093967601B3F7A7009395F501B3E7D700D9
:102B7C0033E5B70067800000930710009306000050
:102B8C0013F7F70013064000E304C7F893874700D8
:102B9C006FF01FF8930700006FF09FF91306050004
:102BAC001305000093F61500638406003305C50079
:102BBC0093D5150013161600E39605FE67800000EA
:102BCC006340050663C605061386050093050500DC
:102BDC001305F0FF630C060293061000637AB6002F
:102BEC006358C0001316160093961600E36AB6FEDF
:102BFC001305000063E6C500B385C5403365D500F9
:102C0C0093D6160013561600E39606FE6780000056
:102C1C0093820000EFF05FFB1385050067800200D4
:102C2C003305A04063D80500B305B0406FF0DFF961
:102C3C00B305B04093820000EFF01FF93305A040BC
:102C4C00678002009382000063CA0500634C050094
:102C5C00EFF09FF71385050067800200B305B040C5
:102C6C00E35805FE3305A040EFF01FF63305B040E6
:102C7C0067800200B7070100637AF5029307F00F33
:102C8C00B3B7A70093973700130700023307F74039
:102C9C00B357F500170500001305C56FB307F50012
:102CAC0003C507003305A740678000003707000104
:102CBC0093070001E36AE5FC930780016FF0DFFCEA
:102CCC00411106C6EFD0CFD4B240B70710F023A005
:082CDC0007F20145410182806D
:102CE4004448525953544F4E452050524F47524135
:102CF4004D2C20534F4D4520535452494E4700000C
:102D04004468727973746F6E652042656E63686D92
:102D140061726B2C2056657273696F6E20322E318E
:102D240020284C616E67756167653A20432900006D
:102D340050726F6772616D20636F6D70696C65644A
:102D440020776974682027726567697374657227D0
:102D540020617474726962757465000050726F67E3
:102D640072616D20636F6D70696C6564207769743E
:102D7400686F75742027726567697374657227209C
:102D8400617474726962757465000000506C6561E9
:102D94007365206769766520746865206E756D6259
:102DA4006572206F662072756E73207468726F7519
:102DB4006768207468652062656E63686D61726B14
:102DC4003A200000457865637574696F6E207374EA
:102DD400617274732C2025642072756E732074687C
:102DE400726F756768204468727973746F6E650AD0
:102DF40000000000457865637574696F6E20656E28
:102E04006473000046696E616C2076616C7565734D
:102E1400206F6620746865207661726961626C65F2
:102E240073207573656420696E207468652062651B
:102E34006E63686D61726B3A00000000496E745FE6
:102E4400476C6F623A202020202020202020202060
:102E54002025640A000000002020202020202020BB
:102E640073686F756C642062653A20202025640ABB
:102E740000000000426F6F6C5F476C6F623A202065
:102E840020202020202020202025640A000000008B
:102E940043685F315F476C6F623A20202020202016
:102EA400202020202025630A00000000202020206C
:102EB4002020202073686F756C642062653A20209E
:102EC4002025630A0000000043685F325F476C6F8F
:102ED400623A202020202020202020202025630A60
:102EE400000000004172725F315F476C6F625B38B3
:102EF4005D3A2020202020202025640A00000000C4
:102F04004172725F325F476C6F625B385D5B375D45
:102F14003A2020202025640A0000000020202020E0
:102F24002020202073686F756C642062653A20202D
:102F3400204E756D6265725F4F665F52756E7320C9
:102F44002B203130000000005074725F476C6F62B8
:102F54002D3E000020205074725F436F6D703A2044
:102F640020202020202020202025640A00000000AA
:102F7400202020202020202073686F756C6420623C
:102F8400653A20202028696D706C656D656E7461EA
:102F940074696F6E2D646570656E64656E74290066
:102FA400202044697363723A2020202020202020AE
:102FB400202020202025640A000000002020456EE7
:102FC400756D5F436F6D703A2020202020202020F3
:102FD4002025640A000000002020496E745F436FBE
:102FE4006D703A2020202020202020202025640AF3
:102FF4000000000020205374725F436F6D703A200C
:1030040020202020202020202025730A00000000FA
:10301400202020202020202073686F756C6420629B
:10302400653A2020204448525953544F4E4520506D
:10303400524F4752414D2C20534F4D45205354522B
:10304400494E47004E6578745F5074725F476C6FE9
:10305400622D3E00202020202020202073686F75E0
:103064006C642062653A20202028696D706C656D5F
:10307400656E746174696F6E2D646570656E6465E8
:103084006E74292C2073616D652061732061626FF9
:1030940076650000496E745F315F4C6F633A20209F
:1030A40020202020202020202025640A0000000069
:1030B400496E745F325F4C6F633A202020202020D9
:1030C400202020202025640A00000000496E745F3F
:1030D400335F4C6F633A20202020202020202020C2
:1030E4002025640A00000000456E756D5F4C6F6317
:1030F4003A20202020202020202020202025640A7F
:10310400000000005374725F315F4C6F633A2020FB
:1031140020202020202020202025730A00000000E9
:10312400202020202020202073686F756C6420628A
:10313400653A2020204448525953544F4E4520505C
:10314400524F4752414D2C2031275354205354524F
:10315400494E47005374725F325F4C6F633A2020CC
:1031640020202020202020202025730A0000000099
:10317400202020202020202073686F756C6420623A
:10318400653A2020204448525953544F4E4520500C
:10319400524F4752414D2C2032274E442053545213
:1031A400494E47004D656173757265642074696D9D
:1031B4006520746F6F20736D616C6C20746F206F69
:1031C400627461696E206D65616E696E6766756CA7
:1031D40020726573756C747300000000506C656137
:1031E400736520696E637265617365206E756D62C7
:1031F4006572206F662072756E730000436C6F6396
:103204006B206379636C65733D2564200A000000BC
:10321400444D49505320706572204D687A3A2020FD
:10322400202020202020202020202020202020209A
:10323400202020202020202020202020000000000A
:1032440025642E00256400004448525953544F4EBF
:10325400452050524F4752414D2C20312753542082
:10326400535452494E4700004448525953544F4E08
:10327400452050524F4752414D2C2032274E442076
:10328400535452494E4700004448525953544F4EE8
:10329400452050524F4752414D2C20332752442051
:1032A400535452494E47000034E2FFFF48E1FFFF08
:1032B40054E1FFFF48E1FFFF20E2FFFF48E1FFFF89
:1032C40054E1FFFF34E2FFFF34E2FFFF20E2FFFF9F
:1032D40054E1FFFF20E1FFFF20E1FFFF20E1FFFFBA
:1032E4005CE1FFFFF0E7FFFFF0E7FFFF14E8FFFFFB
:1032F400E4E7FFFFE4E7FFFFD4E8FFFF14E8FFFF84
:10330400E4E7FFFFD4E8FFFFE4E7FFFF14E8FFFF73
:10331400E0E7FFFFE0E7FFFFE0E7FFFFD4E8FFFFA0
:1033240048EBFFFF84EBFFFF90EBFFFF84EBFFFF15
:10333400FCEBFFFF84EBFFFF90EBFFFF48EBFFFF8D
:1033440048EBFFFFFCEBFFFF90EBFFFF60EBFFFFA1
:1033540060EBFFFF60EBFFFF98EBFFFF88EEFFFFE2
:1033640088EEFFFF08EFFFFF80EEFFFF80EEFFFF18
:1033740068EFFFFF08EFFFFF80EEFFFF68EFFFFF3E
:1033840080EEFFFF08EFFFFF7CEEFFFF7CEEFFFF08
:103394007CEEFFFF68EFFFFF00010202030303035B
:1033A40004040404040404040505050505050505D1
:1033B40005050505050505050606060606060606B1
:1033C4000606060606060606060606060606060699
:1033D4000606060606060606070707070707070781
:1033E4000707070707070707070707070707070769
:1033F4000707070707070707070707070707070759
:103404000707070707070707070707070707070748
:103414000707070707070707080808080808080830
:103424000808080808080808080808080808080818
:103434000808080808080808080808080808080808
:1034440008080808080808080808080808080808F8
:1034540008080808080808080808080808080808E8
:1034640008080808080808080808080808080808D8
:1034740008080808080808080808080808080808C8
:1034840008080808080808080808080808080808B8
:083494000808080808080808F0
:1034A0000000000080842E41000000205FA0124236
:0C34B000F90295503353DE470000C8427B
:040000058000000077
:00000001FF
